:020000040000FA
:1000000005280000000000008B1397018501860180
:100010008B01A701A801A901AA01AC0107309F002B
:1000200083160313E730810030308500C830860026
:10003000831203139820D021A820861D20280611A2
:100040008614DE21DE2107308101A5018E01061410
:10005000831603130614831203134D208316031310
:100060000610831203136420AA012508A9000108C1
:10007000A800A7015E21861006152C1C46286B20BF
:10008000BA20B320C320802196214828ED20D0211A
:10009000C921C921C9212C141B28A201933086191A
:1000A0002730A300A30F55285D286420A20F5528F0
:1000B000F930A200A20F5A285228AF3086195730C3
:1000C000A200A20F612808000B1D6928A50A0B11C8
:1000D0000800000008008619712123210930BA00A8
:1000E000AB01393084003A08063C031D79282B14F3
:1000F000AB142B1882280008003C031D82282030F6
:10010000122193282B14861D89283A08013C0319D3
:1001100008003030BC0000083C071221AB1C9328BB
:100120002E301221AB10BA0B9628080084037328D6
:10013000861202300C2102300C210C300C210030D0
:100140000C210C300C2100300C2106300C21080051
:10015000861200300C2101300C2108300C210030B7
:100160000C218616080086120C300C2100300C2160
:1001700086160800203012214D30122148301221FD
:100180007A301221080042301221613012216E3083
:100190001221643012213A301221861DD8285530A0
:1001A000122148301221463012212030122108003D
:1001B00056301221D128493012216E30122174306C
:1001C00012213A30122108004530122178301221D4
:1001D000743012213A30122108004830122149307F
:1001E000122120301221643012216530122120307A
:1001F0001221573012214E3012213230122141305B
:1002000012212030122176301221353012212E3069
:1002100012213730122108008500DE210616DE216A
:1002200006120800BC00BD003C0E0F398500DA2123
:100230000616DA2106123D080F398500DA21061666
:10024000DA21061208002030BB000930BA00313034
:1002500084008001BA0B2D292F29840A29294D21D8
:100260003421BB0B2F290800273084000310800D98
:10027000840A800D840A800D840A800D0930BA003A
:1002800031308400800D0310001A03140F308005F4
:10029000BA0B4B290800840A42290930BA003130D0
:1002A00084000008A200043C0318592903302207E7
:1002B0008000BA0B5C290800840A51292808A6008E
:1002C000A401A40A8316031301120000011683126D
:1002D00003130108260203196129A409240AA700AF
:1002E00008000330BB00273084000310800D840A0F
:1002F000800D840A800D840A800DBB0B73290800D1
:10030000831603133230850083120313D6212B1179
:1003100085182B15831603133030850083120313C1
:100320002B1D9429E4200800DB2008001030BE00BB
:1003300012309F008316031331308500831203139C
:10034000DE21BE03A0303E07831603139F008312F5
:100350000313DE211F1BAF29003C031DA1298312BB
:10036000031307309F008316031330308500831278
:1003700003133E08093C031CC329203012213030EE
:100380003E07122108003130122126303E0712218B
:100390000800A201A20FCD290800A30FCD29CA2968
:1003A000F030A400C921A40FD2290800A201A20F95
:1003B000D7290800D621D621D6210800DA21DA2152
:0C03C000DA21DA21DA21DA21DA21080042
:02400E00623F0F
:00000001FF
